:100000000C9466000C9485000C9485000C9485007B
:100010000C9485000C9485000C94C6010C9485000A
:100020000C9485000C9485000C9485000C9485003C
:100030000C9485000C9485000C9485000C9485002C
:100040000C94DF080C9485000C9485000C948500BA
:100050000C9485000C9485000C9485000C949E08EB
:100060000C9485000C9485000C941B060C94850060
:100070000C9485000C9485000C9485000C948500EC
:100080000C9485000C9485000C9485000C948500DC
:100090000C94F4090C94D7050C9485000C948500FD
:1000A0000C9485000C9485000C9481010C948500BF
:1000B0000C9485000C9485000C9485000C948500AC
:1000C0000C9485000C9485000C94850011241FBEAF
:1000D000CFEFD1E2DEBFCDBF18E0A0E0B2E0E8E5AF
:1000E000F0E200E00BBF02C007900D92A836B10706
:1000F000D9F71DE0A8E6B8E001C01D92A336B1070C
:10010000E1F70E946B0D0C942A100C94000089EB0F
:1001100096E2A0E0B0E08093F9099093FA09A093E9
:10012000FB09B093FC091092FD0952E05093FE09BF
:1001300031E03093FF0983E08093000A1092010AB6
:100140001092020A3093030A1092040A1092050AD0
:100150004FEF4093060A20E12093070A3093080AE4
:1001600088E998E090930A0A8093090A10920B0A92
:1001700040930C0A20930D0A30930E0A9093100AB4
:1001800080930F0A2093110A5093120A3093130A96
:100190001092140A08958A3010F48093FD0908958E
:1001A0008A3010F48093FE090895AF92BF92CF92E7
:1001B000DF92FF920F931F93CF93DF936C0180E048
:1001C00090E0F601E80FF91F108201968131910548
:1001D000C1F700E010E098ECA92EB12C23C00E94DA
:1001E000620381E06F2D0E947903C5010197F1F749
:1001F00086E00E94F303282F2F713881832F90E02F
:10020000820F911D8F3F910514F4230F2883F394DF
:1002100021968BE1F81619F7A8950F5F1F4F04364A
:10022000110521F0E6018BE0F82ED9CF80E1DF91B6
:10023000CF911F910F91FF90DF90CF90BF90AF9023
:10024000089581E080936F0880916D088F5F80939F
:100250006D080E946203E091FD0980915409F0E06D
:1002600024E0EE0FFF1F2A95E1F7E80FF11DEC5394
:10027000FD4F82E060810E94790388EE93E0019750
:10028000F1F786E00E94F303682F6F7160937408A2
:1002900086E798E00E945209682F80937508809144
:1002A000760890917708A0917808B09179088093AA
:1002B000700890937108A0937208B09373088091AE
:1002C000FF0990917408813051F48091000A8917D8
:1002D00078F480916E088F5F80936E080EC08091D5
:1002E000000A891728F480916E088F5F80936E084A
:1002F00086E798E070E00E947003A89510926F085E
:1003000008951F920F920FB60F920BB60F92112401
:100310002F933F934F935F936F937F938F939F930D
:10032000AF93BF93EF93FF931092A5001092A40098
:100330000E9421012091220230912302E091FE09C6
:1003400080915409F0E044E0EE0FFF1F4A95E1F779
:10035000E80FF11DEC5DFD4F8081280F311D3093BA
:10036000A9002093A800FF91EF91BF91AF919F91B9
:100370008F917F916F915F914F913F912F910F904E
:100380000BBE0F900FBE0F901F9018951F920F92EB
:100390000FB60F920BB60F9211242F933F934F93EA
:1003A0005F936F937F938F939F93AF93BF93EF93DD
:1003B000FF93A8958FE00E94F303982F80916F0818
:1003C000882309F085C092FF07C086E00E94F303EE
:1003D0008F7180934E097CC093FF7AC0809152093F
:1003E00090915309029799F4E091FD098091540985
:1003F000F0E074E0EE0FFF1F7A95E1F7E80FF11DD2
:10040000EC53FD4F81E060810E94790361C082EE70
:1004100098E062E64FE459E021E539E00E94740477
:1004200080935009882309F453C080915109813089
:1004300009F04EC020917008309171084091720807
:10044000509173088091E2089091E308A091E4082C
:10045000B091E50882179307A407B507C9F5809105
:10046000E6088830A8F5809154098F3088F4E0912F
:10047000FD0980915409F0E064E0EE0FFF1F6A95DA
:10048000E1F7EC53FD4FE80FF11D82E061810CC0F4
:10049000E091FD09F0E054E0EE0FFF1F5A95E1F7FF
:1004A000EC53FD4F82E060810E9479038091E60861
:1004B000873019F410926A080BC082EE98E06091C0
:1004C0004E0940914F0920E00E94A20980935009F3
:1004D000FF91EF91BF91AF919F918F917F916F911C
:1004E0005F914F913F912F910F900BBE0F900FBED8
:1004F0000F901F901895DF93CF9300D000D0CDB709
:10050000DEB788E492E0A0E0B0E089839A83AB8311
:10051000BC83CE01019660E070E044E050E00E94B0
:10052000121089EF99E064E070E04CE150E00E9425
:1005300012100F900F900F900F90CF91DF910895B0
:10054000EF92FF920F93DF93CF93CDB7DEB768970B
:100550000FB6F894DEBF0FBECDBF19821A821B8280
:100560001C820E948700CE01019660E070E044E0AA
:1005700050E00E94021089819A81AB81BC81E5E044
:10058000EE2EF12CEC0EFD1E88549240A040B0409F
:10059000D1F489EF99E064E070E04CE150E00E9412
:1005A000021080E092E00E94D2072091F909309178
:1005B000FA094091FB095091FC09C701B90140E0DB
:1005C00020E001E018C080E192E00E94D20769813A
:1005D0007A81C70140E020E001E00E945F06C70188
:1005E0000E94D20780E292E00E94D207C70168E42D
:1005F00072E040E020E00E945F06C7010E94D2073F
:100600008DE092E00E94D20768960FB6F894DEBFA4
:100610000FBECDBFCF91DF910F91FF90EF90089566
:100620008CE390E090932302809322020E94A00228
:100630008091FD098A3010F48093FD090E949E0389
:10064000E091FD0980915409F0E0A4E0EE0FFF1F56
:10065000AA95E1F7E80FF11DEC53FD4F82E06081B0
:100660000E94790385E06FE040E020E00E941704DB
:100670000E943D030E94990808951092A5001092CF
:10068000A4001092A00085E08093A1008FEF90E07D
:100690009093A9008093A800E2E7F0E08081826057
:1006A00080837894089594B7977F94BFE0E6F0E054
:1006B00090819861908387708860808384B7877FFA
:1006C00084BF0895809154098F3030F4809154098B
:1006D0008F5F8093540902C01092540980E00895FE
:1006E0009C01862FB9010E94CC042C9A2C9880E0A2
:1006F00008951F93182F262F88E06FE140E00E9495
:100700001704812F90E09093530980935209113080
:1007100019F482E066E008C085E060E847E021E087
:100720000E94170482E069E00E94E4038EE06CE01E
:100730000E94E403789480E01F9108950F931F9323
:1007400084E00E94BF030CEF13E0C8010197F1F7AA
:1007500017982C988CE090E00197F1F7179A82E0B7
:1007600068E00E94E403C8010197F1F781E06FE1BE
:1007700040E00E94040480E01F910F9108950F9AB9
:10078000249A95B1936095B994B1976094B92398E0
:1007900090E59CBD9CB59C7F9CBD9DB59E7F9DBDFD
:1007A0002CB5982F9370922B9CBD9DB58695869500
:1007B0008170982B9DBDEAE6F0E080818C6080839B
:1007C00080E28CBBED9A0895806C9FB7F8942898CE
:1007D0008EBD0DB407FEFDCF6EBD0DB407FEFDCF7F
:1007E000289A9FBF08958F7380689FB7F8942898C0
:1007F0008EBD0DB407FEFDCF8EBD0DB407FEFDCF3F
:100800008EB5289A9FBF0895FF920F931F93062FCE
:10081000F42E0E94F303082310E002C015950795FB
:10082000FA94E2F7802F1F910F91FF900895DF92C5
:10083000EF92FF920F931F93D82EF62EE42E022FE5
:100840000E94F3036F2D6095682310E002C0000F33
:10085000111FEA94E2F7F0226F298D2D0E94E40324
:100860001F910F91FF90EF90DF900895CB010895B5
:10087000FC01DA015FB7F894289880E28EBD0DB4D0
:1008800007FEFDCF1EBC0DB407FEFDCF4EB56417AD
:1008900030F1942F20E030E01EBC0DB407FEFDCFF8
:1008A0008EB52827022E2295207F2025032E322F59
:1008B00022952F700226269532272327220F220FFA
:1008C000220F20258083915011F03196E5CF1097AB
:1008D00039F01C92232B21F481E08C9301C04068F5
:1008E000289A5FBF842F0895FF920F931F93CF9391
:1008F000DF938C01EA01D901FFB6F894289880E2D1
:100900008EBD0DB407FEFDCF1EBC0DB407FEFDCF9E
:100910009EB5691708F436C020E030E040E050E0B2
:10092000692F70E01CC01EBC0DB407FEFDCF8EB554
:10093000F801E20FF31F80834827042E4295407F81
:100940004025052E542F42954F7004264695542776
:100950004527440F440F440F40252F5F3F4F261774
:10096000370708F3109729F01C92452B11F481E00A
:100970008C93209741F01EBC0DB407FEFDCF8EB5C1
:10098000888301C09068289AFFBE892FDF91CF919C
:100990001F910F91FF900895982FFB012FB7F894A6
:1009A000289880E68EBD0DB407FEFDCF9EBD0DB428
:1009B00007FEFDCF80818EBD915011F03196F7CFAB
:1009C0000DB407FEFDCF289A2FBF0895FC01DA0170
:1009D0003FB7F894289880E28EBD0DB407FEFDCF96
:1009E0001EBC0DB407FEFDCF2EB56217A0F0922FEE
:1009F0001EBC0DB407FEFDCF8EB58083915011F063
:100A00003196F6CF109741F01EBC0DB407FEFDCF16
:100A10008EB58C9301C02068289A3FBF822F08951D
:100A2000833309F080E0089583E30895E82FF0E030
:100A3000EE0FFF1FE55EF54F20813181C90108955A
:100A4000E82FF0E0EE0FFF1FE55EF54F11821082F8
:100A500008959B01AC01529A53985A9A5B9A64E0AC
:100A6000220F331F441F551F6A95D1F760E072E1D2
:100A70008AE790E00E94960F215030401092CD00FE
:100A80002093CC0080E48093C80088E98093C9005B
:100A900086E08093CA00789408959B01AC01689A1F
:100AA0006998709A719A74E0220F331F441F551F82
:100AB0007A95D1F760E072E18AE790E00E94960FA4
:100AC000215030401092C5002093C40080E48093F0
:100AD000C00088E98093C10086E08093C2007894CA
:100AE0000895FC018091180A8823D1F4F0931A0A22
:100AF000E093190A6093180A20911D0A30911E0A8A
:100B0000808190E08227932790931E0A80931D0A8C
:100B100080818093CE008091C90080628093C9005B
:100B20008091180A8823E1F70895FC018091150A45
:100B30008823D1F4F093170AE093160A6093150AFC
:100B400020911B0A30911C0A808190E08227932714
:100B500090931C0A80931B0A80818093C600809129
:100B6000C10080628093C1008091150A8823E1F75B
:100B70000895DF93CF930F92CDB7DEB78983CE016F
:100B8000019661E00E9495050F90CF91DF91089545
:100B9000DF93CF930F92CDB7DEB78983CE01019655
:100BA00061E00E9471050F90CF91DF9108951F922F
:100BB0000F920FB60F920BB60F9211242F933F9303
:100BC0008F939F93EF93FF93E091190AF0911A0A84
:100BD0003196F0931A0AE093190A31978091180A16
:100BE00081508093180A8091180A882391F080918F
:100BF0001D0A90911E0A2181332727FD3095282751
:100C0000392730931E0A20931D0A81818093CE00DC
:100C100005C08091C9008F7D8093C900FF91EF913D
:100C20009F918F913F912F910F900BBE0F900FBE10
:100C30000F901F9018951F920F920FB60F920BB640
:100C40000F9211242F933F938F939F93EF93FF93D2
:100C5000E091160AF091170A3196F093170AE09383
:100C6000160A31978091150A81508093150A809158
:100C7000150A882391F080911B0A90911C0A21810A
:100C8000332727FD30952827392730931C0A2093D6
:100C90001B0A81818093C60005C08091C1008F7DB1
:100CA0008093C100FF91EF919F918F913F912F9180
:100CB0000F900BBE0F900FBE0F901F901895BF9214
:100CC000CF92DF92EF92FF920F931F93DF93CF9318
:100CD000CDB7DEB72C970FB6F894DEBF0FBECDBFF1
:100CE0006C01FB01B42EE22E77FD02C0FF2408C088
:100CF000F095E195FF4F8DE2D6018C93FF24F3949C
:100D000040E08E010F5F1F4F10C0200F311FCF0139
:100D10006AE070E00E94830F805DD9018C93CF015F
:100D20006AE070E00E94830FFB01242F30E04F5FE8
:100D3000EA30F10554F7020F131F8E2F805DF80182
:100D40008083642FCE01019620E305C0FC01E60FED
:100D5000F11D20836F5FE616C8F76B15B8F3862F79
:100D600090E09E012F5F3F4FF901E80FF91F1082BD
:100D70000197D901A80FB91F019640E050E08C01FE
:100D80002E2D30E07EE214C0C801841B950B821723
:100D9000930729F4F601EF0DF11D7083F394F6012A
:100DA000EF0DF11D8C918083F3944F5F5F4F11978E
:100DB000461750F3F601EF0DF11D1082C6012C9677
:100DC0000FB6F894DEBF0FBECDBFCF91DF911F915C
:100DD0000F91FF90EF90DF90CF90BF9008954F92CA
:100DE0005F926F927F928F929F92AF92BF92CF92BB
:100DF000DF92EF92FF920F931F93DF93CF93CDB7C4
:100E0000DEB72C970FB6F894DEBF0FBECDBF3C0106
:100E10006A017B01422E502E77FD02C099240DC03D
:100E2000F094E094D094C094C11CD11CE11CF11C3E
:100E30008DE2F30180839924939488245E010894C1
:100E4000A11CB11C19C00A0D1B1DC701B6012AE067
:100E500030E040E050E00E94B80F605DF801608330
:100E6000C701B6012AE030E040E050E00E94B80F30
:100E7000C901DA016C017D01082D10E08394FAE0CC
:100E8000CF16D104E104F104F4F6A00EB11E8C2DAE
:100E9000805DF5018083482DCE01019620E305C0D9
:100EA000FC01E40FF11D20834F5F5416C8F7441571
:100EB000B8F3842F90E09E012F5F3F4FF901E80FB8
:100EC000F91F10820197D901A80FB91F019620E0E0
:100ED00030E0BC01052D10E05EE214C0CB01821BA6
:100EE000930B8017910729F4F301E90DF11D50834D
:100EF0009394F301E90DF11D8C91808393942F5FFE
:100F00003F4F1197241750F3F301E90DF11D1082A3
:100F1000C3012C960FB6F894DEBF0FBECDBFCF91A4
:100F2000DF911F910F91FF90EF90DF90CF90BF90D6
:100F3000AF909F908F907F906F905F904F900895AB
:100F4000DC010D900020E9F71197A81BB90B6A2F5F
:100F50000E9495050895EF92FF920F93DF93CF9330
:100F6000CDB7DEB72A970FB6F894DEBF0FBECDBF60
:100F7000BC017E010894E11CF11CC70140E020E0A7
:100F800001E00E945F06C7010E94A0072A960FB6E3
:100F9000F894DEBF0FBECDBFCF91DF910F91FF90D0
:100FA000EF900895DC010D900020E9F71197A81B40
:100FB000B90B6A2F0E9471050895CF92DF92EF92CC
:100FC0000F93DF93CF93CDB7DEB72A970FB6F89480
:100FD000DEBF0FBECDBFAB01BC016E010894C11CCA
:100FE000D11CC60120E000E0EE24E3940E94EF064D
:100FF000C6010E94D2072A960FB6F894DEBF0FBE34
:10100000CDBFCF91DF910F91EF90DF90CF900895FA
:10101000EF92FF920F93DF93CF93CDB7DEB72A976E
:101020000FB6F894DEBF0FBECDBFBC017E010894A1
:10103000E11CF11CC70140E020E001E00E945F06D6
:10104000C7010E94D2072A960FB6F894DEBF0FBEE2
:10105000CDBFCF91DF910F91FF90EF900895109247
:10106000800082EC8093810010928200EFE6F0E035
:1010700080818062808378940895FC018081860F4E
:1010800080830895FC018081819580830895FC010F
:101090008081860F80830895FC0180818195808303
:1010A0000895FC0180819181860F971F9183808331
:1010B0000895FC0180819181909581959F4F918346
:1010C00080830895FC0180819181860F971F918311
:1010D00080830895FC0180819181909581959F4F37
:1010E000918380830895FC01882777FD8095982F50
:1010F0002081318142815381260F371F481F591F9C
:1011000020833183428353830895FC018081918140
:10111000A281B381B095A095909581959F4FAF4FD7
:10112000BF4F80839183A283B3830895279A2F981A
:1011300008952F9A08952F98089508951F920F9259
:101140000FB60F9211242F933F938F939F9380910B
:10115000F609882339F48091F7099091F80996955A
:10116000879502C08091F60986BD8091F70990911C
:10117000F809209165083091660801969093F80966
:101180008093F70901978217930729F41092F809C1
:101190001092F70915BC9F918F913F912F910F905D
:1011A0000FBE0F901F9018958093F60970936608F4
:1011B0006093650882E085BD80E888BD08951F9230
:1011C0000F920FB60F920BB60F9211242F933F93ED
:1011D0004F936F937F938F939F93AF93BF93EF93AF
:1011E000FF936091860070918700809164099091CF
:1011F00065099B01281B390B409166098BE0293B4F
:10120000380730F140936009109266098091F9091E
:101210009091FA09A091FB09B091FC0980937B0B96
:1012200090937C0BA0937D0BB0937E0B81E0809319
:101230007F0B8091930B9091940B01969093940B5C
:101240008093930B82E08093D9078091040A14C0A5
:10125000483090F4E42FF0E0C901880F991F820F05
:10126000931F84599141EE0FFF1FED57F44F918367
:1012700080834F5F409366097093650960936409AA
:10128000FF91EF91BF91AF919F918F917F916F915E
:101290004F913F912F910F900BBE0F900FBE0F906B
:1012A0001F9018959C012F98809161099091620977
:1012B000019690936209809361098091630981305E
:1012C000E9F48091DA078130C9F480915B098823C1
:1012D000A9F08FEF8093810B80915B098093820B43
:1012E00010925B098091820B8533A1F41092820BDE
:1012F0001092DA0783E780935B090CC08091DA07CC
:10130000813041F48091810B8F3F21F41092820B48
:1013100010925B09D901EBE7FBE08CE101900D92A3
:101320008150E1F78091F309860F8093F309809152
:10133000F409882329F08091F40981508093F409FD
:101340008CE10895FC012F9A6093F4094093F5090C
:1013500084818330E9F4A7E5BDE08CE001900D9233
:101360008150E1F781E080935D0980915C0D8032CE
:1013700068F4E0915C0DF0E080915D0D90915E0D60
:10138000EE0FFF1FE95EF24F9183808381E01EC064
:101390008430F1F4A7E5BBE084E201900D92815026
:1013A000E1F780915C0B8C3070F480915C0B90E0E5
:1013B000B5E0880F991FBA95E1F78956944F6FE50C
:1013C0007BE00E94FB0F81E080935D0980935E09C2
:1013D0008CE0089584E693E00E94D2070895F89483
:1013E00080E00E945303FFCF1F920F920FB60F921F
:1013F0000BB60F9211241F932F933F934F935F933C
:101400006F937F938F939F93AF93BF93EF93FF93CC
:101410001091CE0080916C0980936D0980916B09C9
:1014200080936C0990916A0990936B0920916909E6
:1014300020936A0910936909823B41F4953A31F48B
:10144000253621F41B3411F40E94EF094091F20972
:10145000442309F04AC0143471F48091F0098434B3
:10146000D1F51093F109109268091092670981E093
:101470008093F2098EC0133531F48091F0098335E1
:1014800051F581E007C0133741F48091F0098337AB
:1014900011F582E080935C097CC0123539F48091AB
:1014A000F0098235C1F40E94EF0973C0153639F492
:1014B0008091F009853679F40E947B026AC01D365E
:1014C00051F48091F0098D3631F410925B0981E07E
:1014D000809363095EC080915B09882309F059C03D
:1014E00010935B091092F20954C08091F109843481
:1014F00009F04BC010926309209167093091680987
:10150000A12FB0E0E42FF0E04C31C0F4A227B327C4
:10151000B070AA0FBB1FA45FBB4F232F33278D9141
:101520009C91822793279093680980936709E359D8
:10153000F64F10834F5F4093F2092BC0A227B327C9
:10154000B070AA0FBB1FA45FBB4F832F99272D91AB
:101550003C91822793279093680980936709DF0164
:1015600011974EE659E0FD01E40FF51F1083892B1A
:1015700061F42BE73BE0C901BA01AD010E94E70F1E
:1015800081E08093D9078091050A1092F2091092A8
:10159000F1091093F009FF91EF91BF91AF919F91E5
:1015A0008F917F916F915F914F913F912F911F91FB
:1015B0000F900BBE0F900FBE0F901F9018950F93BA
:1015C000FC0101900020E9F73197E81BF90BDB01E2
:1015D0006D917C918E0F9F1F40E020E001E00E9402
:1015E0005F060F9108950F93FC0101900020E9F729
:1015F0003197E81BF90BDB016D917C918E0F9F1FDA
:1016000040E020E001E00E945F060F9108950F93F3
:10161000FC0101900020E9F73197E81BF90BDB0191
:101620006D917C918E0F9F1F40E020E001E00E94B1
:101630005F060F9108950F93DC010D900020E9F7EC
:101640001197A81BB90BFB016081772767FD709587
:101650008A0F9B1F40E020E001E00E945F060F918F
:1016600008950F93FC0101900020E9F73197E81BE2
:10167000F90BDB016C918E0F9F1F70E040E020E0C2
:1016800001E00E945F060F9108958F929F92AF92A2
:10169000BF92CF92DF92EF92FF920F931F93DF934F
:1016A000CF93CDB7DEB7A0970FB6F894DEBF0FBECD
:1016B000CDBF282F19824091560990915509A92F25
:1016C000B0E0FD01E153F84FE081BE2EB40E8091F1
:1016D000120A882319F481E08093120A233309F453
:1016E0006AC0243338F4213309F4ACC0223309F042
:1016F000BCC013C0263329F1283321F0243309F06C
:10170000B4C060C0442311F0415012C0AC52B84F75
:101710008C9181508093560910C0242F30E0AC5238
:10172000B84F8C9190E001972817390724F44F5F48
:101730004093560902C010925609B0905609BE0E49
:1017400094C0AB2DB0E0FD01E45FF94FE081E230E1
:10175000F9F0E33030F4EE23D9F0E13009F085C040
:1017600008C0E430F9F0E430E8F0E53009F07DC07D
:1017700022C0AA0FBB1FAD5DB94FED91FC918081D6
:101780009181A281B3818C509E4FAF4FBF4F4BC010
:10179000AA0FBB1FAD5DB94FED91FC918081918186
:1017A0000A9630C0AA0FBB1FAD5DB94FED91FC91F9
:1017B00080818F5F45C0943010F49F5F46C01092C7
:1017C000550949C0AB2DB0E0FD01E45FF94FE08160
:1017D000E23079F0E33030F4EE2359F0E13009F0F3
:1017E00044C013C0E43021F1E43010F1E530E9F5F4
:1017F00029C0AA0FBB1FAD5DB94FED91FC9180814F
:1018000091810A979183808330C0AA0FBB1FAD5D81
:10181000B94FED91FC9180819181A281B381845F68
:101820009140A040B04080839183A283B3831DC0C8
:10183000AA0FBB1FAD5DB94FED91FC918081815026
:10184000808313C0992321F091509093550903C0D0
:1018500084E08093550910925609E0915509F0E013
:10186000E153F84FB080B09257090B2D10E0209152
:1018700057098091120A90E0820F911D0197081775
:1018800019074CF08091120A2B2D281B822F8F5F95
:101890008093570904C0B21610F4B092570983E937
:1018A00093E00E94D207E0915509F0E0E153F84F30
:1018B000208181E090E0821B9109800F911F0E949E
:1018C000080887E993E00E94D207E0915509F0E00B
:1018D000EC52F84F808190E00E94080889E993E07B
:1018E0000E94D207E0915509F0E0EE0FFF1FEB5385
:1018F000F84F808191810E94D2078BE993E00E948A
:10190000D20780EA93E00E94D207E0915509F0E007
:10191000EE0FFF1FEB53F84F6081718183E29BE074
:101920000E94FB0F00E010E0C801815E954F68EB5C
:1019300073E00E94FB0F065E1F4F31E00430130777
:1019400099F7A09057097E010894E11CF11CFAE177
:101950008F2E912C89C01982BA1429F4C7016AEB21
:1019600073E00E94F00F8601000F111FF801E0598B
:10197000F84F60817181C7010E94F00FC7016CEBC5
:1019800073E00E94F00FF601E45FF94FE081E2306E
:1019900001F1E33028F4EE2351F0E130C1F510C03D
:1019A000E43039F1E430F0F0E53089F52BC00D5D1D
:1019B000194FF80160817181C7010E94F30A27C0A5
:1019C0000D5D194FF80160817181C7010E94DF0A26
:1019D0001EC00D5D194FF80160817181C7010E9421
:1019E000070B15C00D5D194FF80160817181C701AA
:1019F0000CC00D5D194FF80160817181C7010E9413
:101A00001B0B05C0C70165E579E00E94310B8EEB29
:101A100093E00E94D207809157099601281B310953
:101A2000C9010E94080889E993E00E94D207C70112
:101A30000E94D20782EC93E00E94D207809157095E
:101A4000F601E81BF109EA30F1056CF4188EE89D07
:101A5000C001E99D900DF89D900D1124815E954F78
:101A6000B7010E94FB0FA394CA2CDD242091120A17
:101A70008091570990E0820F911DC816D906A4F4F1
:101A800036E13A1588F0E0915509F0E0DF01AC52FB
:101A9000B84F2C91E153F84F808190E0820F911D57
:101AA000C816D9060CF457CF80EA93E00E94D207FB
:101AB000A0960FB6F894DEBF0FBECDBFCF91DF91D9
:101AC0001F910F91FF90EF90DF90CF90BF90AF905C
:101AD0009F908F9008954F925F926F927F928F9216
:101AE0009F92AF92BF92CF92DF92EF92FF920F93AD
:101AF0001F93DF93CF93CDB7DEB760970FB6F894FF
:101B0000DEBF0FBECDBF279A2F982F9A8FEF8093FD
:101B1000F6098FEF90E0909366088093650882E065
:101B200085BD80E888BD80E090E0FC01EE0FFF1FDE
:101B3000ED57F44F11821082019680319105A9F77B
:101B400080E090E0FC01EE0FFF1FE95EF24F118292
:101B50001082019680329105A9F780E090E020E89C
:101B60000FB6F89420936100809361000FBE8091BE
:101B70006600875F80936600399A419A54985C9A10
:101B800060E076E980E090E00E94290585EC93E032
:101B90000E94D20784E693E00E94D20710925F0B66
:101BA00080E090E02EE2FC01A5E0EE0FFF1FAA9579
:101BB000E1F7E956F44F2083118201968C309105AC
:101BC00091F70E942F080E9410038091F9099091CB
:101BD000FA09A091FB09B091FC0980937B0B9093CB
:101BE0007C0BA0937D0BB0937E0B81E080937F0BE9
:101BF000F8EC6F2E712C44244A94EFEF8E2E912C2A
:101C000072E0572E6E010894C11CD11C61E1A62E12
:101C1000B12CAC0EBD1E1092F5091092F40980EDA6
:101C200097E0F3013197F1F70197D9F780915E09B9
:101C3000882331F18091020A8F3F79F09091F50964
:101C40008091020A891748F01092F60988EE93E015
:101C5000909366088093650810C08091010A8F3FB9
:101C600079F09091F4098091010A891748F0409227
:101C7000F609909266088092650855BC80E888BD98
:101C80008091DA07882321F510915B0910925B0996
:101C9000153321F481E08093DA071AC0193419F45E
:101CA00084E693E013C0112399F084E693E00E9448
:101CB000D207812F0E94450B8091140A882341F09E
:101CC0001092140A0E947B0283ED93E00E94D207D7
:101CD00080915C09813079F410925C092F9AC601D9
:101CE0000E94D50081EE93E00E94D207C60160E118
:101CF0000E94710520C080915C098230E9F4109245
:101D00005C092F9AC6010E94D50084EE93E00E94E0
:101D1000D207860189EE93E00E94D207F8018191F3
:101D20008F0190E00E9408080A151B0599F782ECC4
:101D300093E00E94D2072F9880915D09882309F4CF
:101D40006ACF8091130A882309F465CF8091DA075E
:101D5000813009F041C08BEE93E00E94D20787EFFB
:101D60009CE00E94D20782EC93E00E94D20784EFAD
:101D700093E00E94D2078AE090E00E94080889E977
:101D800093E00E94D20787ED9CE00E94D20782EC8C
:101D900093E00E94D20700E010E0EE24FF248EEBD7
:101DA00093E00E94D207C8010E94080889E993E0E5
:101DB0000E94D207C7018956944F0E94D20782EC35
:101DC00093E00E94D2070F5F1F4F80E290E0E80E81
:101DD000F91E0A30110519F710925D0989EF93E099
:101DE0000E94D20700E010E089EE93E00E94D20743
:101DF000F801EE0FFF1FED57F44F808191810E9493
:101E000008080F5F1F4F0031110571F78DEF93E048
:101E10000E94D20700E010E089EE93E00E94D20712
:101E2000F801EE0FFF1FE95EF24F808191810E9461
:101E300008080F5F1F4F0032110571F782EC93E025
:101E40000E94D20783E094E00E94D20780916D083F
:101E500090E00E94080889EE93E00E94D2078091EA
:101E60006E0890E00E94080882EC93E00E94D2077E
:101E700087E094E00E94D207809161099091620905
:101E80000E94080889EE93E00E94D2078091F4092D
:101E900090E00E94080889EE93E00E94D2078091AA
:101EA000F50990E00E94080889EE93E00E94D207AD
:101EB0008091F30990E00E94080889EE93E00E9467
:101EC000D2078091600990E00E94080889EE93E0B3
:101ED0000E94D20780917B0B90917C0BA0917D0B8F
:101EE000B0917E0B0E94080889EE93E00E94D20711
:101EF0008091930B9091940B0E94080882EC93E0E0
:101F00000E94D20788CE97FB092E07260AD077FDBC
:101F100004D049D006D000201AF4709561957F4F07
:101F20000895F6F7909581959F4F0895A1E21A2E96
:101F3000AA1BBB1BFD010DC0AA1FBB1FEE1FFF1F6D
:101F4000A217B307E407F50720F0A21BB30BE40BBD
:101F5000F50B661F771F881F991F1A9469F7609504
:101F60007095809590959B01AC01BD01CF010895BE
:101F700097FB092E05260ED057FD04D0D7DF0AD0D7
:101F8000001C38F450954095309521953F4F4F4FA8
:101F90005F4F0895F6F790958095709561957F4F06
:101FA0008F4F9F4F0895AA1BBB1B51E107C0AA1F6B
:101FB000BB1FA617B70710F0A61BB70B881F991FEA
:101FC0005A95A9F780959095BC01CD010895FB0124
:101FD000DC0102C001900D9241505040D8F70895A5
:101FE000FB01DC010D900020E9F7119701900D92A3
:101FF0000020E1F70895FB01DC0101900D92002023
:10200000E1F70895DC01CB01FC01F999FECF06C090
:10201000F2BDE1BDF89A319600B40D9241505040A6
:10202000B8F70895DC01CB0103C02D910E941D106B
:1020300041505040D0F70895262FF999FECF1FBA8E
:1020400092BD81BD20BD0FB6F894FA9AF99A0FBEE1
:0820500001960895F894FFCFFA
:10205800526561645F53657475703A20000A0D001B
:1020680057726F6E672045454D414749433A2000F6
:102078002F00AA000000000000000000000000007F
:102088000000000000000000000000000000000048
:1020980000000000640064006400640064006400E0
:1020A8006400640009120D0810040B0E02140701E5
:1020B8000F050C0009120D0810040B0E021407017D
:1020C8000F050C000A0A0A0A0A0A0A0A0A0A0A0A70
:1020D8000A0A0A0A141414141414141414141414E0
:1020E800141414141E1E1E1E1E1E1E1E1E1E1E1E30
:1020F8001E1E1E1E646464646464646464646464B0
:1021080064646464000102030405060708090A0BF5
:102118000C0D0E0F0E0F14150C100B191A111612A8
:102128000D171318110C1A150F10130B0E180D1686
:102138001719121414120D0F181316110C1A100B6C
:102148000E15191716130E140F181510190B0C1A53
:10215800120D171115101317120E0C1A0B0F110D63
:10216800161814190E0F14150C100B191A11161233
:102178000D17131819110C1A150B140F1810120E2D
:10218800170D13161613180D170F100B190E12151D
:1021980014110C1A0E17120F110C1A1510160B1415
:1021A80019130D180B0C0D0E0F1011121314151610
:1021B8001718191A0A0D535953494E464F3A7A6956
:1021C800676269742F74782D70706D2F61746D65F6
:1021D8006C2F302E382D3133313030363039393597
:1021E8000A0D004D543A002F003A0020200A0D0035
:1021F8002D2D2D2D2D2D2D2D2D2D2D2D2D2D2D2D07
:102208002D2D2D2D2D0A0D0020003E003D004D45A1
:102218003A000A0D0072636F70656E32342D74785F
:102228000A0D0053657475702D53617665640A0D47
:10223800005353005343414E003B00535953494EFA
:10224800464F3A00524D543A00434856000A0D543E
:10225800454C0041433B004554433B000000C1C08E
:1022680081C1400101C3C003800241C201C6C0064A
:10227800800741C70005C1C581C4400401CCC00C1A
:10228800800D41CD000FC1CF81CE400E000AC1CADA
:1022980081CB400B01C9C009800841C801D8C018CA
:1022A800801941D9001BC1DB81DA401A001EC1DE4A
:1022B80081DF401F01DDC01D801C41DC0014C1D43A
:1022C80081D5401501D7C017801641D601D2C0125A
:1022D800801341D30011C1D181D0401001F0C0302A
:1022E800803141F10033C1F381F240320036C1F64A
:1022F80081F7403701F5C035803441F4003CC1FC1A
:1023080081FD403D01FFC03F803E41FE01FAC03AD9
:10231800803B41FB0039C1F981F840380028C1E809
:1023280081E9402901EBC02B802A41EA01EEC02E49
:10233800802F41EF002DC1ED81EC402C01E4C02439
:10234800802541E50027C1E781E640260022C1E259
:1023580081E3402301E1C021802041E001A0C06069
:10236800806141A10063C1A381A240620066C1A649
:1023780081A7406701A5C065806441A4006CC1AC19
:1023880081AD406D01AFC06F806E41AE01AAC06AD9
:10239800806B41AB0069C1A981A840680078C1B8C9
:1023A80081B9407901BBC07B807A41BA01BEC07E49
:1023B800807F41BF007DC1BD81BC407C01B4C07439
:1023C800807541B50077C1B781B640760072C1B259
:1023D80081B3407301B1C071807041B00050C190A9
:1023E800819140510193C053805241920196C05649
:1023F800805741970055C19581944054019CC05C19
:10240800805D419D005FC19F819E405E005AC19AD8
:10241800819B405B0199C059805841980188C04808
:1024280080494189004BC18B818A404A004EC18E48
:10243800818F404F018DC04D804C418C0044C18438
:10244800818540450187C047804641860182C04258
:10245800804341830041C1818180404001030303DF
:102468000303030303030303030203030303020336
:10247800030303F909FD09FE09FF09000A010A021D
:102488000A030A040A050A060A070A080A090A0BBF
:102498000A0C0A0D0A0E0A0F0A110A120A130A1464
:1024A8000A6964007461626C650074696D657461C1
:1024B800626C65006C697374656E5F6265666F72E5
:1024C800655F74616C6B006C62745F6C696D6974D4
:1024D80000727373695F7761726E696E67006C7101
:1024E800695F7761726E696E670070706D5F696EA3
:1024F8000070706D5F73796E630073657269616CEB
:102508005F73796E63006D756C74695F6368616E83
:102518006E656C006D756C74695F6368616E6E657D
:102528006C73006D756C74695F6D73796E635F6E43
:10253800756D006D756C74695F6D73796E635F6C32
:10254800656E006D756C74695F6368616E6E656C4D
:102558006D6170006D756C7469325F6368616E6E71
:10256800656C006D756C7469325F6368616E6E6569
:102578006C73006D756C7469325F6D73796E635F2F
:102588006E756D006D756C7469325F6D73796E630D
:102598005F6C656E006D756C7469325F6368616E3F
:1025A8006E656C6D6170006D656E755F6C656E0053
:1025B8006373765F6F757470757400736176650008
:1025C800510654065A066406770681068E069A0650
:1025D800A106AA06B606C406D306E306F306040750
:1025E8001307230734074507570760076B07476C2E
:1025F8006F62616C00496E707574004D756C74691A
:1026080070726F70004D756C746970726F70320003
:102618004D656E75009E07A507AB07B507C0070097
:10262800070A0F140703050503020101010101014F
:102638000101010101010101010101010101010182
:102648000101010101010101010101010101010172
:102658000101010101010101010101010101010162
:102668000101010101010101010101010101010152
:102678000101010101010101010101010101010142
:102688000101010101010101010101010101010132
:102698000101010101010101010101010101010122
:1026A8000101010101010101010101010101010112
:0826B8000101010101FF000016
:00000001FF
